:020000040800F2
:10100000EA320E0249464C4947485431000000007C
:101010000000000001010000100008183001640FFA
:10102000001E0000000064000100E803DC05D0079A
:101030006400800C000000000E00000000000000B2
:101040000000646661230000000000000000000052
:101050000000000000000000000000000000000090
:101060000000000000000000000000000000000080
:101070000000000000000000000000000000000070
:101080000000000000000000000000000000000060
:101090000000000000000000000000000000000050
:1010A0000000000000000000000000000000000040
:1010B0000000000000000000000000000000000030
:1010C0000000000000000000000000000000000020
:1010D0000000000000000000000000000000000010
:1010E0000000000000000000000000000000000000
:1010F00000000000000000000000000000000000F0
:1011000000000000000000000000000000000000DF
:1011100000000000000000000000000000000000CF
:1011200000000000000000000000000000000000BF
:1011300000000000000000000000000000000000AF
:0811400000001932000000005C
:1014000000200020C1610008BF610008914400086D
:1014100000000000000000000000000000000000CC
:10142000000000000000000000000000BF61000894
:1014300000000000000000003144000809430008DB
:10144000BD610008BD610008BD610008BD61000804
:10145000BD610008BD610008BD610008BD610008F4
:10146000BD6100086917000811510008413C0008DF
:10147000BD6100080D17000849170008D140000899
:10148000313C0008BD610008BD610008BD61000875
:10149000BD610008BD610008BD610008BD610008B4
:1014A000BD610008BD610008BD61000891500008E1
:1014B000BD610008BD610008BD610008BD61000894
:1014C00001225549554B524270B50A601A600022FC
:1014D0000A601A60524B534A534D1A60534B544A98
:1014E00054481A600322544B54492B60544B8024B7
:1014F0001A60544A6401121A04F05EFB8022524BB7
:1015000092051A60514B524A52491A6022230B60CD
:101510009023514A5148DB0514601860504B5148E4
:10152000186002202E683043286080200D68400239
:1015300028438025086011686D00294311601A68EE
:10154000494910200A4042311A60FF3104F090FEF0
:1015500080211B2004F08CFE40211C2004F088FE1A
:101560008021092004F084FE80210A2004F080FEFE
:1015700040210B2004F07CFE0D2004F06DFE0E20B7
:1015800004F06AFE0F2004F067FE102004F064FEF1
:10159000142004F061FE1B2004F05EFE1C2004F009
:1015A0005BFE092004F058FE0A2004F055FE0B20D3
:1015B00004F052FE10222D4B1A602D4B30321A606F
:1015C0002C4B38321A6080222B4B12061D602B4B9D
:1015D0001C602B4B1A601A68002AFCDB0122294888
:1015E0001A6001681142FBD0274B284A1A60072273
:1015F000274B1A60C022274B12041A60264B274A39
:101600001A600422264B1A70264B274A1A60274A72
:10161000274B1A6070BDC0460C10024010100240EB
:1016200014100240050006001C1002401810024071
:10163000014A00000000002011080000001400080A
:1016400000000140C00000202000004824000048A5
:1016500022020000200400480C040048FFBFEAEB0F
:1016600000040048FAEFFFFFFFFEFFFF082C0140D7
:1016700004000040180000401C0000402000004012
:1016800008240140002401400C2401400104000012
:101690001424014008270140282401404800030089
:1016A000CC0200201000024040240140C002002073
:1016B0001400024003230340013B0022022B01D807
:1016C000044AD256430702D580231B011A43024B1A
:1016D0001A607047AC6200081C000140064B1A6893
:1016E000D20708D4054A1178054A1160054A1A60E4
:1016F0000422054B1A60704708000240CC0200200B
:101700000C00024083050000082401400A4B10B57C
:101710001A68D1070BD5022149421960074B1B6893
:10172000002B04D0064907480B6803400B60930662
:1017300001D502F097FC10BD102C0140402C014057
:101740001C000140FFF8FFFF1122054B52421A60B6
:101750008023044ADB0011680B4313607047C046C6
:10176000102C01401C0001400222F0B500261B4B4A
:101770001B4D1A601B4B1C4F1E601C4B87B01888FA
:10178000E988784304F02EFC194B1A8892B2029231
:10179000184A11888AB2198803928BB204932B8855
:1017A0006C8843431B130593AB883900444358436B
:1017B00004F018FC029B049AC31AA020400058436E
:1017C000039B2413991A04F00DFC23003100059AA1
:1017D0007830009602F0E4FC07B0F0BD040002404F
:1017E000C002002008000240E40C0000BAF7FF1F0E
:1017F000B8F7FF1FC2F7FF1F044B1A68002A04DB6B
:10180000002802DB024A18601060704708020020BE
:101810004002002070B505000E000024A300F0581F
:10182000002804D0290004F0E1F9002801D12000AB
:1018300070BD0134F2E713B50A220C0001A904F0CF
:10184000E1FA03000020019A1278824201D123605C
:10185000013016BD10B50400006804F0BEF9206028
:1018600010BD000030B50D0085B0040064212800D3
:1018700004F0B8FB0A2201A904F08CF90100200051
:10188000FFF7E8FF20000E49FFF7E4FF280064217E
:1018900004F08EFC0A22080001A904F07BF904F090
:1018A000E5F90500012D05DD200001A9FFF7D2FFB4
:1018B00005B030BD20000349FFF7CCFF0135F1E74B
:1018C00080650008826500081FB504000A22080030
:1018D00001A904F05FF901002000FFF7BBFF1FBD65
:1018E000F0B5070000248DB001902500474901A8FC
:1018F00004F0C3F9002804D1002C0BD128000DB04E
:10190000F0BD0378002BF1D0A20002AB0134D0501F
:101910000A2CEAD13E4902980197FFF77BFF09287C
:1019200001D901F04AFB04F0C9FA0A0015009D0034
:10193000AE03E2063E0B4B0B500B6A0B810B354995
:1019400001A8FFF787FF344901A8FFF783FF019B38
:10195000DD1BD3E7012C01D001F02FFB2F4901A89B
:10196000FFF778FF2E4CA078FFF746FF010001A893
:10197000FFF7AAFF2B4901A8FFF76CFFE17801A848
:10198000FFF7A2FF284901A8FFF764FF274901A834
:10199000FFF760FF264901A8FFF75CFF254B01A870
:1019A0001968FFF791FF244C2368002B07D02349C7
:1019B00001A8FFF74FFF216801A8FFF785FF204925
:1019C00001A8FFF747FF1F4B01A81968FFF74AFF5F
:1019D0001D4901A8FFF73EFF1C4B01A81968FFF73E
:1019E00041FF1B4901A8FFF735FF1A4B01A81968F1
:1019F000FFF76AFF184901A8FFF72CFF174B01A852
:101A00001968FFF761FF16499AE7C0468465000828
:101A1000F867000889650008BC670008F1650008E0
:101A2000C000002080650008FE650008C40000209A
:101A300001660008C8070020CC0700200A660008DD
:101A400012660008E80700201B6600087C070020DB
:101A500024660008780700202D6600088C07002007
:101A600087650008012C01D001F0A7FAFB4901A805
:101A7000FFF7F0FEFA4D01A82900FFF7EBFEF94E43
:101A800001A8317DFFF720FFF74C01A82100FFF7E7
:101A9000E1FEF64901A8FFF7DDFE290001A8FFF7E6
:101AA000D9FE717D01A8FFF70FFF210001A8FFF704
:101AB000D1FEEF4901A8FFF7CDFE290001A8FFF7ED
:101AC000C9FEB17D01A8FFF7FFFE210001A8FFF7C5
:101AD000C1FEE84901A8FFF7BDFE290001A8FFF7F4
:101AE000B9FEF17D01A8FFF7EFFE210001A8FFF785
:101AF000B1FEE14901A8FFF7ADFE290001A8FFF7FB
:101B0000A9FE317E01A8FFF7DFFE210001A8FFF743
:101B1000A1FEDA4901A8FFF79DFE290001A8FFF701
:101B200099FE717E01A8FFF7CFFE210001A8FFF703
:101B300091FED34901A8FFF78DFE290001A8FFF708
:101B400089FEB17E01A8FFF7BFFE210001A8FFF7C3
:101B500081FECC4901A8FFF77DFE290001A8FFF70F
:101B600079FEF17E01A8FFF7AFFE210001A8FFF783
:101B700071FEC54901A8FFF76DFE290001A8FFF716
:101B800069FE317F01A8FFF79FFE210001A8FFF742
:101B900061FEBE4901A8FFF75DFE290001A8FFF71D
:101BA00059FE717F01A8FFF78FFE210001A8FFF702
:101BB00051FEB74901A8FFF74DFE290001A8FFF724
:101BC00049FEB17F01A8FFF77FFE210001A8FFF7C2
:101BD00041FEB04901A8FFF73DFE290001A8FFF72B
:101BE00039FEF17F01A8FFF76FFE210001A8FFF782
:101BF00031FEA94901A8FFF72DFE290001A8FFF732
:101C000029FE731CD97F01A8FFF75EFE210001A801
:101C1000FFF720FEA14901A8FFF71CFE290001A83B
:101C2000FFF718FE9E4B01A8D97FFFF74DFE21005C
:101C300001A8FFF70FFE9B4901A8FFF70BFE290043
:101C400001A8FFF707FEF31CD97F01A8FFF73CFEB0
:101C5000210001A8FFF7FEFD934901A8FFF7FAFD57
:101C6000290001A8FFF7F6FD331DD97F01A8FFF772
:101C70002BFE210001A8FFF7EDFD8C4901A8FFF71D
:101C8000E9FD290001A8FFF7E5FD731DD97F01A833
:101C9000FFF71AFE210001A8FFF7DCFD844901A827
:101CA000FFF7D8FD290001A8FFF7D4FDB31DD97FA8
:101CB00001A8FFF709FE210001A8FFF7CBFD7D4930
:101CC00001A8FFF7C7FD290001A8FFF7C3FDF31D19
:101CD000D97F01A8FFF7F8FD210001A8FFF7BAFDA1
:101CE000754901A8FFF7B6FD290001A8FFF7B2FD6D
:101CF00033000833D97F01A8FFF7E6FD210001A8D2
:101D0000FFF7A8FD6D4901A8FFF7A4FD290001A870
:101D1000FFF7A0FD33002833197801A8FFF7D4FDA1
:101D2000210001A8FFF796FD654901A8FFF792FD84
:101D3000290001A8FFF78EFD718D01A8FFF7C4FDF2
:101D4000210001A8FFF786FD5E4901A8FFF782FD8B
:101D5000290001A8FFF77EFDB18D01A8FFF7B4FDB2
:101D6000210001A8FFF776FD574901A8FFF772FD92
:101D7000290001A8FFF76EFDF18D01A8FFF7A4FD72
:101D8000210001A8FFF766FD504901A8FFF762FD99
:101D9000290001A8FFF75EFD318E01A8FFF794FD31
:101DA000210001A8FFF756FD494901A8FFF752FDA0
:101DB000290001A8FFF74EFD718E01A8FFF784FDF1
:101DC000210001A8FFF746FD424901A8FFF742FDA7
:101DD000290001A8FFF73EFD33003433197801A82C
:101DE000FFF772FD210001A8FFF734FD3A4901A871
:101DF000FFF730FD290001A8FFF72CFD3300353334
:101E0000197801A8FFF760FD210001A8FFF722FD66
:101E1000324901A8FFF71EFD290001A8FFF71AFDAE
:101E200033003633197801A8FFF74EFD210001A8D1
:101E3000FFF710FD2A4901A8FFF70CFD290001A8B2
:101E4000FFF708FD33003733197801A8FFF73CFD91
:101E5000210001A8FFF7FEFC44E0C04638660008F8
:101E600035660008C0000020876500083C66000851
:101E7000416600084866000850660008576600087A
:101E8000626600086D660008766600087F660008D6
:101E900088660008916600089B660008A566000831
:101EA000C2000020AF660008B9660008C3660008DB
:101EB000CE660008D8660008E2660008EC660008F6
:101EC000F6660008006700080A6700081467000843
:101ED0001F6700082A670008356700084067000888
:101EE0004B670008DB4901A8FFF7B4FC290001A8F3
:101EF000FFF7B0FC33003833197801A8FFF7E4FC92
:101F0000210001A8FFF7A6FCD34901A8FFF7A2FC16
:101F1000290001A8FFF79EFC718F01A8FFF7D4FCF0
:101F2000210001A8FFF796FCCC4901A8FFF792FC1D
:101F3000290001A8FFF78EFC33003C33197801A873
:101F4000FFF7C2FC210001A8FFF784FCC44901A8E7
:101F5000FFF780FC290001A8FFF77CFC33003D332C
:101F6000197801A8FFF7B0FC210001A8FFF772FC67
:101F7000BC4901A8FFF76EFC290001A8FFF76AFC25
:101F800033003E33197801A8FFF79EFC210001A819
:101F9000FFF760FCB44901A8FFF75CFC290001A829
:101FA000FFF758FC33003F33197801A8FFF78CFC8A
:101FB000210001A8FFF74EFCAC4901A8FFF74AFC3D
:101FC000290001A8FFF746FCA94B01A8D98FFFF70C
:101FD0007BFC210001A8FFF73DFCA64901A8FFF703
:101FE00039FC290001A8FFF735FCA34901A8FFF738
:101FF00031FC210001A8FFF72DFCA04901A8FFF743
:1020000029FC290001A8FFF725FCA1235B00F15C56
:1020100001A8FFF759FC210001A8FFF71BFC984914
:1020200001A8FFF717FC290001A8FFF713FC4423C0
:10203000FF33F15C01A8FFF747FC210001A8FFF77F
:1020400009FC904901A8FFF705FC290001A8FFF74A
:1020500001FCA2235B00F15C01A8FFF735FC210025
:1020600001A8FFF7F7FB884901A8FFF7F3FB290058
:1020700001A8FFF7EFFB4623FF33F15C01A8FFF750
:1020800023FC21005CE4022C01D000F096FF7F4984
:102090000398FFF7BFFB292801D900F08EFF7C4C85
:1020A0007C4D03F00BFF2A003F00520065007800D2
:1020B0008B009E00B100C4000D01200133014601D8
:1020C00051015C01670172017D01880193019E014C
:1020D000B201C501D801EB01FE0111021C02270269
:1020E00032023D0248025B02660271027C028702F4
:1020F0009B02A802BD02C9021903674901A8FFF7A4
:10210000A9FB290001A8FFF7A5FB644D01A8297DC3
:10211000FFF7DAFB01A82100FFF79CFB287DFFF702
:102120006BFB10E45E4901A8FFF794FB290001A8AE
:10213000FFF790FB594D01A8697DFFF7C5FB01A88A
:102140002100FFF787FB687DE9E7564901A8FFF703
:1021500081FB290001A8FFF77DFB504D01A8A97D57
:10216000FFF7B2FB01A82100FFF774FBA87DD6E7BB
:102170004D4901A8FFF76EFB290001A8FFF76AFB94
:10218000464D01A8E97DFFF79FFB01A82100FFF75D
:1021900061FBE87DC3E7454901A8FFF75BFB290028
:1021A00001A8FFF757FB3D4D01A8297EFFF78CFBE7
:1021B00001A82100FFF74EFB287EB0E73C4901A8AB
:1021C000FFF748FB290001A8FFF744FB334D01A8A6
:1021D000697EFFF779FB01A82100FFF73BFB687ED2
:1021E0009DE7344901A8FFF735FB290001A8FFF757
:1021F00031FB2A4D01A8A97EFFF766FB01A821004B
:10220000FFF728FBA87E8AE72B4901A8FFF722FBEE
:10221000290001A8FFF71EFB204D01A8E97EFFF76A
:1022200053FB01A82100FFF715FBE87E77E7234960
:1022300001A8FFF70FFB290001A8FFF70BFB174DC3
:1022400001A8297FFFF740FB01A82100FFF702FB4F
:10225000287F64E756670008626700086D6700081A
:1022600077670008816700088B6700089667000899
:10227000C2000020A067000802010020A667000835
:10228000AD670008B4670008B86700082468000854
:10229000876500083566000838660008C000002021
:1022A0003C66000841660008486600085066000861
:1022B00057660008626600086D66000876660008CA
:1022C000E34901A8FFF7C6FA290001A8FFF7C2FAFF
:1022D000E04D01A8697FFFF7F7FA01A82100FFF799
:1022E000B9FA687F1BE7DC4901A8FFF7B3FA2900B8
:1022F00001A8FFF7AFFAD74D01A8A97FFFF7E4FACD
:1023000001A82100FFF7A6FAA87F08E7D34901A892
:10231000FFF7A0FA290001A8FFF79CFACD4DE97F4D
:1023200001A8FFF7D1FA01A82100FFF793FAE87F8F
:10233000F5E6CB4901A8FFF78DFA290001A8FFF7C0
:1023400089FAC44D0135EAE7C64901A8FFF782FAC8
:10235000290001A8FFF77EFABE4D0235DFE7C2492A
:1023600001A8FFF777FA290001A8FFF773FAB94D22
:102370000335D4E7BD4901A8FFF76CFA290001A88D
:10238000FFF768FAB34D0435C9E7B94901A8FFF76B
:1023900061FA290001A8FFF75DFAAE4D0535BEE7E9
:1023A000B44901A8FFF756FA290001A8FFF752FA2D
:1023B000A84D0635B3E7B04901A8FFF74BFA29004D
:1023C00001A8FFF747FAA34D0735A8E7AB4901A8D5
:1023D000FFF740FA290001A8FFF73CFA9D4D0835A8
:1023E0009DE7A74901A8FFF735FA290001A8FFF7E3
:1023F00031FA984D2835297801A8FFF765FA01A828
:102400002100FFF727FA287889E69E4901A8FFF7FF
:1024100021FA290001A8FFF71DFA8E4D01A8698D48
:10242000FFF752FA01A82100FFF714FA688D76E64B
:10243000954901A8FFF70EFA290001A8FFF70AFA4B
:10244000844D01A8A98DFFF73FFA01A82100FFF7ED
:1024500001FAA88D63E68D4901A8FFF7FBF9290071
:1024600001A8FFF7F7F97B4D01A8E98DFFF72CFADA
:1024700001A82100FFF7EEF9E88D50E6844901A894
:10248000FFF7E8F9290001A8FFF7E4F9714D01A869
:10249000298EFFF719FA01A82100FFF7DBF9288E32
:1024A0003DE67C4901A8FFF7D5F9290001A8FFF70F
:1024B000D1F9684D01A8698EFFF706FA01A821003D
:1024C000FFF7C8F9688E2AE6734901A8FFF7C2F939
:1024D000290001A8FFF7BEF95E4D34358BE76F493F
:1024E00001A8FFF7B7F9290001A8FFF7B3F9594D83
:1024F000353580E76A4901A8FFF7ACF9290001A842
:10250000FFF7A8F9534D363575E7664901A8FFF77F
:10251000A1F9290001A8FFF79DF94E4D37356AE76B
:10252000614901A8FFF796F9290001A8FFF792F980
:10253000484D38355FE75D4901A8FFF78BF9290061
:1025400001A8FFF787F9434D01A8698FFFF7BCF990
:1025500001A82100FFF77EF9688FE0E5544901A842
:10256000FFF778F9290001A8FFF774F9394D3C35D8
:1025700041E7504901A8FFF76DF9290001A8FFF7CD
:1025800069F9344D3D3536E74B4901A8FFF762F94B
:10259000290001A8FFF75EF92E4D3E352BE747498C
:1025A00001A8FFF757F9290001A8FFF753F9294DB2
:1025B0003F3520E7424901A8FFF74CF9290001A85F
:1025C000FFF748F9234D01A80235E98FFFF77CF9A1
:1025D00001A82100FFF73EF9E88FA0E501A83949DD
:1025E000FFF738F9290001A8FFF734F9364901A8A7
:1025F000FFF730F945E5354901A8FFF72BF9290028
:10260000A12501A8FFF726F9124E6D00715D01A802
:10261000FFF75AF901A82100FFF71CF9705D7EE56C
:102620002B4901A8FFF716F92900442501A8FFF757
:1026300011F9084EFF35E9E7264901A8FFF70AF925
:10264000290001A8FFF706F9A225024EDDE7C046E2
:102650007F660008C00000208866000891660008B8
:102660009B660008A5660008AF660008B96600080A
:10267000C3660008CE660008D8660008E266000857
:10268000EC660008F6660008006700080A670008A4
:10269000146700081F6700082A67000835670008EC
:1026A000406700084B67000856670008626700082B
:1026B0006D67000877670008816700088B6700086E
:1026C00096670008A067000802010020A6670008BE
:1026D000AD670008B4670008D94901A8FFF7BAF848
:1026E000290001A8FFF7B6F84625D64EA2E7032C2D
:1026F00001D000F062FCD4490398FFF78BF8292839
:1027000001D900F05AFC03F0D9FB2A004900680007
:102710008600A400C200E000FF001E013D015C0134
:102720007B01BD01CC01DB01EA01F90108021702BE
:1027300026023502550274029302B202D102F0025F
:10274000FF020E031D032C033B035A0369037803A6
:10275000BB03CA03EA030104210430043F046946B1
:102760000498FFF768F8002801D100F026FC009BD0
:10277000B44C237502F072FEB44901A8FFF76AF861
:10278000B34901A8FFF766F8217D01A8FFF79CF87F
:1027900001A8B049FFF75EF8207DC0E469460498BF
:1027A000FFF749F8002801D100F007FC009BA54C79
:1027B000637502F053FEA84901A8FFF74BF8A4493E
:1027C00001A8FFF747F8617D01A8FFF77DF801A890
:1027D000A049FFF73FF8607DA1E469460498FFF740
:1027E0002AF8002800D1E8E3009B964CA37502F07C
:1027F00035FE9A4901A8FFF72DF8954901A8FFF782
:1028000029F8A17D01A8FFF75FF801A89149FFF71A
:1028100021F8A07D83E469460498FFF70CF80028AE
:1028200000D1CAE3009B874CE37502F017FE8C4988
:1028300001A8FFF70FF8864901A8FFF70BF8E17D23
:1028400001A8FFF741F801A88249FFF703F8E07DEE
:1028500065E469460498FEF7EEFF002800D1ACE37A
:10286000009B784C237602F0F9FD7E4901A8FEF723
:10287000F1FF774901A8FEF7EDFF217E01A8FFF7E0
:1028800023F801A87349FEF7E5FF207E47E4694677
:102890000498FEF7D0FF002800D18EE3009B694C1E
:1028A000637602F0DBFD704901A8FEF7D3FF6849AB
:1028B00001A8FEF7CFFF617E01A8FFF705F801A888
:1028C0006449FEF7C7FF607E29E469460498FEF775
:1028D000B2FF002800D170E3009B5A4CA37602F0AF
:1028E000BDFD624901A8FEF7B5FF594901A8FEF7F1
:1028F000B1FFA17E01A8FEF7E7FF01A85549FEF749
:10290000A9FFA07EFFF70BFC69460498FEF793FF32
:10291000002800D151E3009B4A4CE37602F09EFD73
:10292000534901A8FEF796FF494901A8FEF792FF17
:10293000E17E01A8FEF7C8FF01A84649FEF78AFF1D
:10294000E07EFFF7ECFB69460498FEF774FF002871
:1029500000D132E3009B3B4C237702F07FFD4549D9
:1029600001A8FEF777FF3A4901A8FEF773FF217F20
:1029700001A8FEF7A9FF01A83649FEF76BFF207FEB
:10298000FFF7CDFB69460498FEF755FF002800D1FC
:1029900013E3009B2B4C637702F060FD364901A8DE
:1029A000FEF758FF2A4901A8FEF754FF617F01A8EE
:1029B000FEF78AFF01A82749FEF74CFF607FFFF76B
:1029C000AEFB69460498FEF736FF002800D1F4E21A
:1029D000009B1C4CA37702F041FD284901A8FEF79B
:1029E00039FF1B4901A8FEF735FFA17F01A8FEF7BB
:1029F0006BFF01A81749FEF72DFFA07FFFF78FFBA4
:102A000069460498FEF717FF002800D1D5E20D4C67
:102A1000009BE37702F022FD194901A8FEF71AFF97
:102A20000B4901A8FEF716FFE17F01A8FEF74CFF56
:102A300001A80849FEF70EFFE07FFFF770FBC046D4
:102A4000B8670008C0000020246800083866000845
:102A500035660008876500083C6600084166000886
:102A6000486600085066000857660008626600085D
:102A70006D660008766600087F66000888660008B4
:102A80009166000869460498FEF7D5FE002800D13B
:102A900093E2E14C009B0134E37702F0DFFCDF4975
:102AA000BBE769460498FEF7C6FE002800D184E221
:102AB000D94C009B0234E37702F0D0FCD849ACE754
:102AC00069460498FEF7B7FE002800D175E2D24CA3
:102AD000009B0334E37702F0C1FCD2499DE76946CD
:102AE0000498FEF7A8FE002800D166E2CA4C009BBD
:102AF0000434E37702F0B2FCCB498EE769460498D0
:102B0000FEF799FE002800D157E2C34C009B053424
:102B1000E37702F0A3FCC5497FE769460498FEF716
:102B20008AFE002800D148E2BB4C009B0634E377C4
:102B300002F094FCBE4970E769460498FEF77BFEFC
:102B4000002800D139E2B44C009B0734E37702F04F
:102B500085FCB84961E769460498FEF76CFE0028D9
:102B600000D12AE2AC4C009B0834E37702F076FCFB
:102B7000B14952E769460498FEF75DFE002800D18E
:102B80001BE2A54C009B2834237002F067FCAB4984
:102B900001A8FEF75FFEAA4901A8FEF75BFE2178B7
:102BA00001A8FEF791FE01A8A649FEF753FE207882
:102BB000FFF7B5FA69460498FEF73DFE002800D1FC
:102BC000FBE1009B944C638502F048FC9E4901A800
:102BD000FEF740FE9A4901A8FEF73CFE618D01A870
:102BE000FEF772FE01A89749FEF734FE608DFFF7ED
:102BF00096FA69460498FEF71EFE002800D1DCE133
:102C0000009B854CA38502F029FC904901A8FEF7A2
:102C100021FE8B4901A8FEF71DFEA18D01A8FEF73C
:102C200053FE01A88749FEF715FEA08DFFF777FA3E
:102C300069460498FEF7FFFD002800D1BDE1009B26
:102C4000754CE38502F00AFC814901A8FEF702FEFB
:102C50007B4901A8FEF7FEFDE18D01A8FEF734FED9
:102C600001A87849FEF7F6FDE08DFFF758FA6946AE
:102C70000498FEF7E0FD002800D19EE1009B664C21
:102C8000238602F0EBFB734901A8FEF7E3FD6C49D4
:102C900001A8FEF7DFFD218E01A8FEF715FE01A8B1
:102CA0006849FEF7D7FD208EFFF739FA6946049888
:102CB000FEF7C1FD002800D17FE1009B564C6386E2
:102CC00002F0CCFB644901A8FEF7C4FD5C4901A8F1
:102CD000FEF7C0FD618E01A8FEF7F6FD01A8594977
:102CE000FEF7B8FD608EFFF71AFA69460498FEF702
:102CF000A2FD002800D160E1474C009B34342370D2
:102D000002F0ACFB554943E769460498FEF793FD92
:102D1000002800D151E1404C009B3534237002F073
:102D20009DFB4F4934E769460498FEF784FD00286F
:102D300000D142E1384C009B3634237002F08EFB08
:102D4000484925E769460498FEF775FD002800D13B
:102D500033E1314C009B3734237002F07FFB424952
:102D600016E769460498FEF766FD002800D124E1C5
:102D7000294C009B3834237002F070FB3B4907E775
:102D800069460498FEF757FD002800D115E1009B25
:102D9000214C638702F062FB354901A8FEF75AFD1A
:102DA000274901A8FEF756FD618F01A8FEF78CFDAB
:102DB00001A82449FEF74EFD608FFFF7B0F9694680
:102DC0000498FEF738FD002800D1F6E0124C009B75
:102DD0003C34237002F042FB2649D9E66946049848
:102DE000FEF729FD002800D1E7E00B4C009B3D34A5
:102DF000237002F033FB2049CAE669460498FEF7C7
:102E00001AFD002800D1D8E0034C009B3E3423700B
:102E100002F024FB1949BBE6C00000209B660008B5
:102E2000A5660008AF660008B9660008C36600081A
:102E3000CE660008D8660008E2660008EC66000866
:102E40003566000887650008F66600080067000818
:102E50000A670008146700081F6700082A6700084F
:102E600035670008406700084B6700085667000890
:102E7000626700086D6700087767000881670008CF
:102E800069460498FEF7D7FC002800D195E06E4C07
:102E9000009B3F34237002F0E1FA6C4978E6694602
:102EA0000498FEF7C8FC002800D186E0664C009B21
:102EB0000234E38702F0D2FA654901A8FEF7CAFCA2
:102EC000644901A8FEF7C6FCE18F01A8FEF7FCFCEF
:102ED00001A86149FEF7BEFCE08FFFF720F98022D0
:102EE0005E4C52000499200002F09AFE02F0B6FAFD
:102EF00001A85B49FEF7AEFC01A85649FEF7AAFC03
:102F0000210001A8FEF7A6FCFEF77DFD69460498A6
:102F1000FEF791FC002850D0A1244B4D009B64008B
:102F20002B5502F09BFA4F4901A8FEF793FC494943
:102F300001A8FEF78FFC295D01A8FEF7C5FC01A8DA
:102F40004549FEF787FC285DFFF7E9F869460498D4
:102F5000FEF771FC002830D044243B4D009BFF3429
:102F60002B5502F07BFA4049DEE769460498FEF7EC
:102F700062FC002821D0A224334D009B64002B5515
:102F800002F06CFA3949CFE769460498FEF753FC22
:102F9000002812D046242C4D009BFF342B5502F004
:102FA0005DFA3349C0E7012C07D102F0EDFBFEF7D3
:102FB00023FC002801D0FEF7C6FC2E49FEF7C4FC16
:102FC000012CFAD102F038FCF1E7A31E012BF4D852
:102FD000A1231D4A5B00D35C0093032C04D000990D
:102FE000039802F053FCE4E769460498FEF723FCDB
:102FF0000028E2D0009B013B632BF0D9DDE7022CD7
:10300000DBD169460398FEF716FC0028D5D0FA22DA
:10301000009BD2009918FA2212019142CDD8164A8B
:1030200013600022154B1A70FEF78DFC012CC4D1E1
:10303000134B1A68002A01DA00221A601A68114B31
:103040001A60FEF780FCC046C00000208B670008B5
:1030500096670008356600088765000802010020B1
:10306000A0670008A6670008AD670008B4670008FD
:10307000B8670008C0670008D00700205807002084
:10308000080200204002002000231149114A124882
:1030900010B50B60136003601048114C0360114BB6
:1030A0001C602024104B1C60104B24340360012052
:1030B0000F4B4042186001230E4803600E48046025
:1030C0000E48113C04600B6080239B00136010BD10
:1030D000200400400C04004004040040440002406E
:1030E000E80200205000024048000240A305000012
:1030F0002C04004014040040080400401804004060
:1031000010B50D4B1B78002B01D0FFF7BDFF00223F
:103110000A4B02211A600A4B85321A60094B494258
:103120001A88094B1A600123084A1360084A116083
:10313000084A136010BDC046280300204400024026
:1031400000040040E40200202C040040140400406D
:10315000100400400C040040F8B5574C2368022BC3
:1031600043D0042B00D1A1E0012B19D102225348F6
:10317000534D544E5242026037682A68BA4224DAEC
:1031800051480468A446614601340460002908D10E
:103190004E4B9A5C4E4B1A6001235B424D4A1360C2
:1031A000F8BD092C06DC4A48026813405210013B66
:1031B0000260F3E70132974203D02A6000230360E4
:1031C000ECE700232B603360F8E74425424A41498D
:1031D0001560424A143D15600522524202600932D0
:1031E00022603F4A0A603F4AD9E70323334D5B42DE
:1031F0002B603D4B34481968102319400368344A4A
:103200005E1C0660002B06D1002902D08021374BBE
:1032100019600023C3E71368092E07DC5810002942
:1032200001D11060BCE780230343B8E7244E326825
:10323000002902D02E498A4202D180272B490F60F3
:103240000521494229600931216000210160082BD4
:1032500001D07F2B04D1002AA2D0013A32609FE72F
:103260001A48511C31608354022907D10278002A80
:1032700004D14278FF2A01D102F0E6FF0A2B00D0E8
:103280008EE7002545543560FEF72AFB0D4B18608C
:10329000A84200D184E7104B124A1D600D4B1D60FF
:1032A000012313600D4A1360236079E70722034B63
:1032B00052421A600223F7E70C0400401004004059
:1032C0002C03002038070020440700203003002092
:1032D000D0020020340400400804004020040040D4
:1032E000710200001404004010040048002C00404B
:1032F000FF03000070B5384B1C68384B28331B782F
:10330000002B59D0364B374AE318934225D9364B18
:10331000364AE318934220D9354B364AE318934294
:103320001BD9354B354AE318934216D9344B354AED
:10333000E318934211D9344BF03AE31893420CD975
:10334000324B503AE318934207D9314BE318EE2B36
:1033500003D9304BE3189E2B2ED820002E4B2F4A3A
:10336000F5301A602E49FF3002F03CFEFA239B0034
:1033700058432C4A2C4913680019C0180B680324C1
:1033800001330B6019001060214023420BD1274B01
:10339000274C1D68A84207DD4042206001201160D3
:1033A000404201F0E5FF70BD2468A04204DA4042CB
:1033B000186011600120F4E71E4B1F4A1A601F4B72
:1033C0001F4A1A6031221F4B1A601F4B363A1A608F
:1033D0001E4B09321A60E6E734040040C0000020AA
:1033E0007FADFFFFDE060000FFB4FFFF3E060000DA
:1033F000BFD6FFFF6E0300007FDAFFFF1E03000051
:10340000FFE1FFFF7E0200003FEDFFFFFFF0FFFF47
:10341000BFF4FFFF7FF8FFFF00300040AAAA0000C2
:1034200018FCFFFF4807002040070020500700203D
:103430005407002034070020193600081804004003
:103440009192000020040040100400400C04004051
:103450005049F8B50A68012314001C401A4233D0C1
:10346000022252420A604C4A1068102204001440A2
:10347000104202D1494B1C60F8BD49480268013234
:1034800002600F2AF8DD474A4748442510600022B1
:103490004648474C02602560464C474D2560302425
:1034A00004600520404208604449093008604449EE
:1034B0000A60444A44491160444A45491160454AFA
:1034C0001360454A1360D7E7344B404E1A6835689D
:1034D000501C1860002ACFD04049414F2A000F608D
:1034E00037490F68002F1FD0FA22D200954205DD20
:1034F0002C4B3C4A1A60FFF7FDFEBDE70A682F2AF5
:1035000000D105240C600121324A116000221A60AA
:10351000B2E75210013C3B2AFBDC334A1168A1425E
:1035200004D014600122F2E70224F4E7002CA3DBAC
:103530000328A1DD2D491B4BA1402D4A2D4F1A60B8
:103540002D4A2E4B48101A60C01902F04BFD2C4931
:103550002C4BA140013885B248101D80C01902F0E3
:1035600041FD0022284B01381880104B1A60104B87
:1035700044321A600F4B113A1A6001230F4A13604C
:10358000104A1560134A1360204B214A1E60214BDC
:10359000BDE7C04610040040100400483C0700206E
:1035A000D4020020340700205931000820040040D4
:1035B0000804004018040040783200000C04004069
:1035C000280400402C040040E104000034040040C2
:1035D000710200001404004000040040003000406C
:1035E000CCCC0000F5320008E0020020F0490200D7
:1035F000B5360008006CDC023937000830070020BF
:10360000D8B80500E4020020E60200204C00024089
:10361000E80200205000024037B5FA251C4B1D4A35
:103620001B68ED001068AB4209DB03001C3B042B58
:1036300006D8194B194A1A600122194B1A7037BD66
:10364000AF22184BD200C3189342F8D8124B134A3A
:10365000154C1A60631DDB7F002B15D0A18D0A006D
:10366000323A904209DA0023618D00930F4B01F04A
:10367000B5FE03000E4A1360E1E7002332318842B1
:10368000F8DDE28D0095F2E7618D3231F7E7C04653
:10369000340400403804004000300040AAAA000072
:1036A000C5070020E0FCFFFFC000002030F8FFFF4E
:1036B000D00700200123154A1168194224D014496B
:1036C0000868184220D0022040420860114908686A
:1036D000002806D10B6010210F4B1B680B400F49CF
:1036E0000B7020210E4B19600E4B0F491960012100
:1036F0000E4B494219600E4B023119600D4B80315F
:10370000196080239B0013607047C0460C04004082
:10371000100400402004004010040048280300204A
:103720004800024044000240A30500002C04004071
:103730001404004000040040AC4A10211068F8B5A1
:1037400003000B4008424DD0FFF79EFCA8490B68D0
:10375000002B13D1A74AA84814680200002C03D0FC
:103760002200844200DD02008020800001E052102F
:1037700001338242FBDA5B0213430B600A681300D9
:103780001001121127D10F252C009C4313009B4FD1
:103790000443260098000641300005265E43284079
:1037A000385C0133B0400243042BF2D101240125DF
:1037B00093480F33644216001E412E4200D0E4436A
:1037C00044800230013BF6D28E4A1368002B04D1AC
:1037D00000230B60F8BD5340D3E7013B1360002B7F
:1037E000F6D0F7E7884D2978002928D07824874932
:1037F00087480B6003608748036004608648703C1C
:1038000004607F4C8548136004601724844804607A
:1038100084481060844A136072B6844B1A68844BE3
:103820009B1A132B00DA1323824A83481360012367
:10383000036000688148008810600B6062B6002257
:1038400014007F4B7F48198801318B104788060090
:1038500064009F4201DB01273C430232202A1BD136
:10386000210022002B7809111DD1002B00D0D2435A
:103870000F2113000B400A4212D1734A73491160A1
:10388000102261112240002900D170E12F2910DDA2
:10389000002A00D172E16CE1B68804308E42D5DB9B
:1038A000FFF72EFC96E74A40DDE72F235B1A5B000B
:1038B00073E1002A00D18DE74E4B1B68002B00D02E
:1038C00088E7634A634C1068884201D01160236026
:1038D0002368092B01DC013323601368581E2E284E
:1038E00000D977E702F0E0FA2F002F002F002F0019
:1038F0002F0076FF32003A0041004A0076FF520066
:103900005B00690076FF76FF76FF76FF76FF730037
:103910007B00C400D300DF0076FFCC00D900E500B7
:1039200076FF76FF76FF76FF76FF76FF76FF76FFEF
:1039300076FF76FF76FFEB0000011501290176FF87
:1039400076FF76FF3C01444A137043E72368062B59
:1039500000D03FE70022414B9A753BE72368062BD6
:1039600000D037E701223D4BF6E72368062B00D055
:1039700030E70022394B0533DA772BE72368062B33
:1039800000D027E7354B01220533F5E72368062BE6
:1039900000D01FE701F0F8FE314B18601AE72368EA
:1039A000062B00D016E701222E4B1A70E022104B96
:1039B00012011A600A22134BF3E02368062B00D091
:1039C00008E70022274B1A70094B274AF1E72368C2
:1039D000062B00D0FEE60022244B1A70FAE623687C
:1039E000062B00D0F6E60122204BF6E74400024009
:1039F000880700209007002080FF0000D0680008A2
:103A00000C0200204C070020280300202004004066
:103A10000804004018040040040400405000024024
:103A20004800024093050000340400402404004094
:103A30009F0500002C04004014040040E602002012
:103A4000E4020020E802002000300040AAAA0000A2
:103A5000D8020020DC02002059070020C00000200E
:103A60004002002084070020FF0E00009507002080
:103A7000462201234C49FF32885C03438B54A9E65C
:103A8000462201204849FF328B5C8343F6E74622F9
:103A90004549FF320223885CEFE746224249FF3264
:103AA00002208B5CF1E746223F49FF320423885C09
:103AB000E3E746223C49FF3204208B5CE5E72368BC
:103AC000062B00D086E6384902330A7E52080132BE
:103AD0000F2A03D81300082A00DA08235A000A76AE
:103AE000073B324A136075E62368062B00D071E667
:103AF0002D49CA7E920801320C2A03D81300062AE7
:103B000000DA0623DAB29000D200C8760A77053BC5
:103B1000E7E72368062B00D05CE6234C0A21631CF0
:103B2000D87F02F0D5F90130C0B20A2800D90020B0
:103B30000A2343430134E3772EE72368062B00D0A2
:103B400048E6194C0A21A31CD87F02F0C1F90130C4
:103B5000C0B20A2800D901200A2302344343EAE70D
:103B60002368062B00D035E601F066FE14E7002A34
:103B700013D001200E4A107000290ED00A4B0533D5
:103B8000DA7F0B002F3B002A07D08323DB0099420A
:103B900000DA8AE6074BC9184B00074A1360002277
:103BA000064B1A6016E6C046C00000204002002006
:103BB000C5070020E9FBFFFFD0070020D802002046
:103BC000104B114A03211A608022104B12021A6016
:103BD00054220F4B1A600F4B233A1A600E4B303AA7
:103BE0001A600E4B19600E4B2C3119600D4B303999
:103BF00019600D4B053119600C490A6084321A6056
:103C00007047C04634070020513400084404004087
:103C10000804004018040040200400400C04004048
:103C2000280400402C04004000040040140400401C
:103C300010B5024B1B68984710BDC04634070020E2
:103C4000802210B5034B92011A60034B1B68984702
:103C500010BDC04604000240300700200122014B85
:103C60001A60704714100040F8B5AF4BAF4C1D6898
:103C7000AF492368002D00D171E00120AD4A1560E5
:103C8000AD4A1560AD4AAE4D10602A78002A05D1C4
:103C9000002B03D03C3253433B3B23600A7823681C
:103CA000002A0FD0013B002B09DD236023685A1E38
:103CB0001E00772A0DDCEF36773318000EE0B423B0
:103CC0005B00F2E7B422013352009342EDDD0123A1
:103CD000EBE71800793EF138EF2AEDDD99499A4B70
:103CE0000C6878219B7E091BDB008B4200DD0B00FA
:103CF00083249649964F0C60964C52002760964C50
:103D0000964F125B76005A43D2111A323A60325BF8
:103D1000934E5A43D2111A3240003260025B534331
:103D2000904ADB111A33136081230B602C78002C2E
:103D300014D18D4B8D4A20001A6068228C4B1A607A
:103D40008C4B8D4A1A6021228C4B1A608C4B1C6064
:103D5000FDF7B0FC8B4B1C6001232B70F8BD09787C
:103D600000297FD0013B002B7ADD23602668864B3B
:103D700001209B19013B1B780640DA1017009A437B
:103D80001F408E4200D004253E00064007426FD0FF
:103D90006D4B5B7D002B00D0052680237B485B01AB
:103DA0003343022637426CD0C021C901084366491B
:103DB0004E36497D002900D1403E33431900042688
:103DC00037426BD0604B5A7D531E9A4193020133A8
:103DD000FF33664A0B4364496D4E0860644930689E
:103DE0000A60644A1360FDF765FCFA233560694D8B
:103DF000694E28681B0198425BDD684A1360002306
:103E00003360674B00201E6880236649664ADB05E5
:103E1000632E69DC0860A221C901116085221A6045
:103E20000022624B29681A60554B11321A602368D0
:103E30005F4A013B9B009950524B1B68052B00DCED
:103E40008CE7136851685B1891685B18D1685B1840
:103E5000116952695B189B18514ADB1013607DE7AA
:103E6000062382E70133062B00DC7EE701237CE793
:103E7000024203D105434F4B4F4892E74D4B4F4809
:103E80008FE740211943324203D0A023DB011843BE
:103E900095E78023DB011843354390E78023DB005F
:103EA0000B43324203D103221543454A93E7454A67
:103EB00091E7336801333360062BA2D1374F3B685B
:103EC000181A01F045FE2B685B10984209DD0023AB
:103ED0002C4A13603C4A13703C4B314A2B603C4BDC
:103EE00013602B683B608AE7C72E02DC0860E22182
:103EF00092E791273F02BC46FA27BF00BE4202DA92
:103F00000860614689E7FA27FF00BE4205DA0860CB
:103F1000614611608622FF3281E780204000086000
:103F2000614611602B4A7AE7B8070020BC070020E1
:103F3000B5070020340000402C0000401400004071
:103F4000AC07002080070020C0000020002C0140AA
:103F5000CF0700002C2C0140B0620008342C014037
:103F6000382C01403C2C0140182C014068680000AE
:103F70001C2C0140202C014055050000142C014050
:103F80000C000040C0070020B26A0008680800006A
:103F9000A80700209C07002074070020E4070020E9
:103FA00090070020402C01401C0000401000004001
:103FB0005C070020041000004808000058080000BA
:103FC000486800005868000094070020204E000058
:103FD00000E1F5058502000070B501F03DFC184ECA
:103FE000184D3368184C002B0BD02B78002B08D0C1
:103FF00020683C211D3001F0F5FF0130062815DC5A
:104000002060002333602B70104B1B78002B10D0E6
:10401000FFF72AFE21220E4B00201A60FDF74AFB13
:104020000C4B22681A600023236070BD01232360BB
:10403000E7E7094B094A1A606822094B1A60E9E769
:10404000B8070020AC070020BC070020A007002014
:10405000142C0140A4070020182C014068680000BF
:104060001C2C0140144B70B51B689B0622D5134CC9
:104070007021236812481D0002680D40402D00D1B8
:104080008B43E0218025C9011940ED01A94201D1EE
:104090000C490B40702115000D40402D00D18A4382
:1040A000236002602022084B1A60084B413A1A60D4
:1040B000FFF7DAFD70BDC0460C2C0140182C014002
:1040C0001C2C0140FF8FFFFF142C0140102C0140DD
:1040D00001202749274A0B6870B51468034211D0A4
:1040E00004420FD002235B4213600023224A0B607C
:1040F0001360224A1370224B224A1A60224B234A31
:104100001A6070BDDB06FCD5214B1D4D1B682A686B
:1041100050109842F5DC032042439010984203DC93
:10412000002054109C4207DAFA24174E012036680A
:10413000E400A64200DB00209B18104C9B10154A9F
:104140002B602070127E5A4352119B1A5A10012B79
:1041500000DC0122104B1A600122104B1A60002370
:10416000054A0B601368052BCBDC01331360C8E7ED
:104170000C00004010000040C00700209407002001
:104180009C070020409C00009007002000E1F505FE
:1041900040000040C00000203400004014000040F7
:1041A000F7B5444C0100256817005E1B424B00D553
:1041B0006FE001221A700A22404801F021F98310B1
:1041C000DA43D21713403E4A0021136004000A224A
:1041D0003C4801F015F98310DA433B49D217794383
:1041E00013403A4A4914136005000722384801F089
:1041F00007F93849384B714318600422C91237480F
:1042000001F0FEF8364A1060364A11684318364904
:10421000136008688005810D00280AD133489B127D
:10422000066811609B1903605B2043433048DB1331
:104230000360304E33003C331B78002B11D032002A
:104240003D3212789B00E81A012A05D0022A28D0B4
:10425000E01A002A00D05842002827DA0020264B16
:104260001860264B1B78002B12D005220899244891
:1042700001F0C6F83300FA240833DA7F1423E4008F
:104280005343318E728E009401F0A8F81D4B1860D4
:10429000F7BD1A78002A02D176107619266000261A
:1042A00089E7AC4200DA2C00E01AD5E73C28D6DDDD
:1042B0003C20D4E758020020B40700204C02002024
:1042C000C807002050020020E4320200CC07002082
:1042D000540200200C300000E807002048020020B3
:1042E0007C07002098070020D8070020B007002096
:1042F00078070020C0000020800700205807002019
:1043000044020020D007002080220D4B52051A6085
:1043100000220C4B1A600C4A13780133DBB21900EF
:1043200013700F221140134209D1084A1368013358
:104330001360074A1268934201D1064B1970704707
:1043400004ED00E010ED00E0D4070020D8070020C5
:10435000E0070020DC07002070B503000C0072B6F7
:10436000074A084D1068C018074B186001232B70CE
:1043700062B62B78002B00D170BDA047F9E7C0468C
:10438000D8070020DC070020E0070020F0B5224C11
:104390008DB02378002B0BD044222049FF32895C5A
:1043A000013B1F4A9B00985801F070FA00232370CC
:1043B0001C4E3468002C1CDBA123184A5B00D35C24
:1043C0000193192B01DA19230193002502AF200074
:1043D0000A2101F0EDFE200002C70A2101F002FED1
:1043E0000135041EF3D1FA272B007F005C1E02D298
:1043F00034600DB0F0BD9D4203D038000A49FFF78C
:10440000ABFF02AAA300D358084A9B009858019911
:1044100001F03CFA2300E9E759070020C000002022
:1044200058690008400200205D3C0008B86A000896
:1044300070B5114C2378002B06D0104B1D78002D41
:1044400002D100F071FE25700D4B1B781B0712D1B5
:10445000FDF744F90B4B1B68DB0601D100F0A0FE11
:104460004623094AFF33D05C084B1A68824202D0C7
:10447000186000F05FFF70BDC5070020C407002072
:10448000D4070020D8070020C00000203C020020F4
:10449000012010B500F04EFF80220C4B02211A6063
:1044A0000B4B0C4A49421A600B4B0C4A1A60012311
:1044B0000B4A13600B4A11600B4A0B3111601168F3
:1044C0001942FCD18022094B1A60FEE7142C0140EE
:1044D00028100040BF1200002C1000400F270000E1
:1044E000141000401010004000100040002C00404C
:1044F000F0B5B348B34A99B0B349121A01F05CFB66
:1045000000F0ACFFB14C0025E37D0993231DDA7F59
:10451000AF4B1A7023000833DA7F14235343AD4A9C
:104520001360230036331A78AB4B1A70FCF7C8FFC0
:1045300000F0DAFE00F0DAFE00F03EFDFFF740FB8F
:10454000A64BA74AA7491A60A74BA84AFE201360AA
:104550008123A74A13603522A64B1A60A64B303A36
:104560001A60A64B013A1D602C3B1A60033A0A60A0
:1045700084321A60802101F07BFE0721A04BA14A02
:104580001360A14A1560A14A116022003F321278DF
:104590000B930A929E4A1378002B00D1E7E00A9B06
:1045A000002B08D1DC219B4B49001868B830FF3044
:1045B00001F018FD0A908022974B52041D681A6082
:1045C000C0232E00DB051E401D421DD120004230BD
:1045D00003787E2B00D0D1E0904801F0BDFA011E97
:1045E00000DBC6E031008E4801F012FA23003E33B2
:1045F0001B78002B08D08B4B0A9AFA208A491A6044
:10460000FFF7AAFEFFF7C2FE237D002B01D16B004E
:1046100021D5864B864A874C1A60874B874A884F3C
:104620001A6001220423874E23606A4D9B183A606A
:104630002360073B33602A6001223368134200D1B4
:10464000A2E00023614A2B6023604333FF33D15C37
:104650007D4801F01BF9FFF7BFFC142200210DA8D3
:1046600001F0B3FA32230C93FA2314229B000021A9
:1046700013A80E9301F0A9FAC82300255B0012933A
:10468000C833149300232E000793049303930693D7
:10469000023305934D4F6D48F97E01F0A3FC6C4B3E
:1046A000069A002408909A4201D04A4B1C68797EF1
:1046B00014274F433B005A1E93410A215B42194085
:1046C0002B005A1E93415B42404A1E40002C00D0F2
:1046D000CCE0059B012B01D1013305933C4B043207
:1046E000D27F1978914207D00999002904D11A7014
:1046F000002D01D1FFF770FC354B1B78002B4DD0FE
:104700006424544B1868314B241A0333DB7F9C42DA
:1047100000DD1C0000252E4B1A781A23002A07D131
:104720001300002D04D0294A527D002A00D01A33EC
:104730000999089A002900D0483A0092FA220021EB
:10474000D200200000F04AFE8323294A0899136012
:10475000264B1960404B1860404B1860404B186066
:1047600081231360002D00D1A6E22600C3E030BFF4
:1047700011E7642800DC36E7642134E7A1235B00FD
:10478000E15C01F083F831E730BFFFF7FFFD2B68F4
:10479000002B00D150E701233B604DE7314A1268FE
:1047A000052A06DDC822304992000968914200DBE3
:1047B000FFE11424054B0333D87F4443AAE7C046E6
:1047C000C00000200802002000100008C0000020E7
:1047D000A0070020D0070020C4070020442C01407F
:1047E0001A88000014000040CF0700002C2C014064
:1047F000002C0140042C0140280000402C00004007
:10480000B70B000014E000E018E000E010E000E06A
:10481000B4070020E8070020241002400301002014
:10482000F46E0008400200205D3C000828100040A3
:10483000BF120000001000402C100040C30900000F
:104840001410004010100040E068000880BB000019
:10485000B80B000080070020342C0140382C0140A8
:104860003C2C0140C00700208C070020002C00DBFE
:10487000D4E0531DDB7F022B00D0BBE0059B022B55
:1048800000D0BAE0931DD87F937D04385A4253413B
:10489000D24A44431278A4105340D14A1370D14BEA
:1048A0001A680B00002A00D14B42DB19CE48A34204
:1048B00000DBBCE01422437F807F534342430092DD
:1048C000FA222000C919D20000F088FD0400C54B6F
:1048D0001A68002A00D16EE1002C00D0BDE0C34B65
:1048E0001968002907D02D215143C148196001F0F2
:1048F00079FBC04B1860C04B01271A68002A23D1EE
:10490000099ABE4C002A00D1B4E1B54AB64B1278E0
:104910005B7D002A00D155E1002B00D158E1B84958
:104920005823B84AB84801270260B84A1360B84B08
:10493000B14A196021232360A94B1B78013313600E
:104940009622AA4B92001A600222B24B1A6030BF24
:10495000B14B1A780F23110019401A4248D1069B17
:104960000B9A934200DDC7E19F4B3E331A780A9BB6
:104970005A430A235343A94A1268934200DCBFE119
:10498000069B01330693984B598F002900D1BFE154
:10499000A34801F027FBA34BC218A34B0CA819682E
:1049A000891000F041FD039B00141B18039300D4F1
:1049B000A8E1002303938C4B0233DA8F002A00D145
:1049C000A8E164235A43994B12A8196800F02CFD02
:1049D000049B80121B180493DB43049ADB171A40D4
:1049E000FA230492DB009A4200DD0493FFF7CEFC29
:1049F0003D004FE6032B00D044E71421D31D0332C2
:104A0000D27FDB7F4A434B4320000092884900223B
:104A100000F0E4FC0123040005937BE6937D6F4ADC
:104A2000127853406E4A13700023059337E77F1ABC
:104A3000418F00290ED07F4801F0D4FAFA2300906C
:104A40001B0120003A00002100F0C8FC654B002447
:104A500018603CE791208000F0E772B6764B1B7837
:104A6000002B23D0644B3C211E68013E300001F036
:104A7000B9FA5B4B05001B78002B00D14CE10135E6
:104A8000062D00D100253C21300001F091FB0131C1
:104A9000544B6A4A1E686A4B71431960694B136034
:104AA0000123694AED181360534B1D6000254D4BDF
:104AB000664E1D60604B1D70654B1D60654B1D7023
:104AC000594B1E60FFF7D0F862B6310000260CA8E3
:104AD00000F0A6FC03950135099B002B08D0404B44
:104AE000454A1B78116801338B4201D000231360C3
:104AF000039B049A9F1A3F19FB43DB171F403B4B54
:104B00001968002912D03A4801F06CFA394B0400B8
:104B10001860354B5048197F01F064FA089B0090EB
:104B20004E4A20004E4900F059FC089014212E4AAC
:104B30003048D37F01324B43D17FFA2292004A435F
:104B4000FA21C90000910068002100F047FC454BA4
:104B500004001A6819235B425343FA22D2009B18BF
:104B6000BB4200DD3B009C4200DD1C00394B1A7843
:104B700000239A4202D11C4B0233DB7F0721DA105B
:104B80000B4007998B4200DD0132079B01330793ED
:104B9000082B01D100230793B4420EDA2C4B1B687B
:104BA000052B00DCB7E5B61AB44200DDB3E53400EE
:104BB000B1E5039390E701258EE7B618B44200DA19
:104BC000A9E5F4E7002B05D027496823274AA9E681
:104BD0002749A5E64221FF31F7E7C04695070020A7
:104BE000B5070020B8070020C00000209007002073
:104BF000008793038C070020BC070020142C014081
:104C00005404000058680000182C01401C2C01407E
:104C1000202C014010ED00E0D4070020E807002020
:104C2000002D3101E0FCFFFF9C0700207C070020E5
:104C300030F8FFFF54581400AC0700202C0000404F
:104C400034000040FFFF030014000040409C0000BF
:104C5000C00700209407002080BB000060EA00002D
:104C600030750000800700204505000068580000EE
:104C70001404000072B62B4A2B4D12681A602B4B9D
:104C80002B4A1D602B4B1A60FEF7EEFF21232A4AA8
:104C90002360116810330B431360284B284A1360BC
:104CA000284A1360284B1F6062B629000CA800F048
:104CB000B7FB099B039347E6244B26001F68002F90
:104CC00000D141E672B631211B4A13688B43136051
:104CD0001F4B1D4A1D601B4B1D6001231360FFF716
:104CE0007BF91C4B1D601C4B1D70124B1D601B4B38
:104CF0001D6062B62F0027E6002F00D043E688E44F
:104D0000069140E6039BA02B00DC54E6A02351E66D
:104D1000039150E6049269E63C214143891B3C31F2
:104D2000B6E6C046A4070020409C00009C07002077
:104D300000E1F505900700200C2C0140FFFF030067
:104D4000340000402C00004014000040BC0700204C
:104D50000C000040C0070020940700208C070020B2
:104D60000A4A30B5FF230400121A08001840121A2C
:104D700006200D122B40D31A054A13711B12D57051
:104D8000107054709170537130BDC046F9FF00002F
:104D9000EC070020036810B5D41823121B19DBB2EE
:104DA000036013007D3B0748012B06D820239A435C
:104DB0000B685C1C0C607D24C4540B685C1C0C608C
:104DC000C25410BDEC07002037B5002305000C00CD
:104DD000684601A9102200930193FFF7DBFFEAB2B6
:104DE000684601A9FFF7D6FF2A12684601A9D2B288
:104DF000FFF7D0FF6846E2B201A9FFF7CBFF22120E
:104E0000684601A9D2B2FFF7C5FF2214684601A97E
:104E1000D2B2FFF7BFFF6846220E01A9FFF7BAFF23
:104E2000009B6846DA4301A9D2B2FFF7B3FF0198AD
:104E30003EBD000070B5042850D1294A1378042BD8
:104E40004CD1D378917854781B020B43254A1B1917
:104E5000934243D1244A130037331978062301398A
:104E60005B424B430F2121405B185D1E052D35D859
:104E70002109092904D00A2909D008292ED170BD99
:104E80001A4B6D00E95A2000FFF76AFFF7E7981EFA
:104E9000042804D800F0FEFF080D10121400144B73
:104EA0001B6828335943EEE7124B0A211B6828334D
:104EB000F8E7114B1968E6E7104BFBE7104BF9E7F1
:104EC0003832104B11781868490801F08BF88023AC
:104ED00001005B029842D6DB0B49D4E70020CEE705
:104EE000EC070020FBFF0000C0000020E46A00087F
:104EF000C8070020CC070020E80700207C0700201E
:104F0000780700208C070020FFFF0000030010B589
:104F10000020022B30D11E4B1A787E2A2CD15978D2
:104F20001F2319401B4B1A0037321278013A914265
:104F300022D119490A68062A00D108600A68174870
:104F40005400245A501C08600020052A14D8100070
:104F500000F0A0FF0306080A1315114B196808E0BA
:104F6000104BFBE7104BF9E7104B1968CD23594361
:104F7000C9122000FFF728FF10BD0D4BEEE73833B4
:104F800019780C4B4908186801F02CF80100F0E77B
:104F9000EC070020C000002004080020F06A000890
:104FA000C8070020CC070020E80700207C0700206D
:104FB000780700208C070020A223224AFF331360C9
:104FC000214B1978214B03290DD0042933D0022914
:104FD0001CD11F4A0A311A601E4A116080211E4AE4
:104FE0000904116012E01D491D4819601D49116036
:104FF0001A21184A11608321174A090411600268B6
:1050000019491140802292010A4302601968174A27
:10501000174B002911D0C82111601D221A60154BB1
:10502000154A16491A60164B164A1360164A116043
:10503000164A136070477321D3E788211160092253
:10504000ECE7C0460C380140C4070020FC070020F4
:10505000354E000814380140043801400D4F000857
:105060000C04004841030000FFCFFFFF0838014057
:1050700000380140380002402438014028380140FF
:10508000EC0700203C0002402400024028000240BF
:10509000F7B5154C40252368144E1A002A4001929A
:1050A0002B4218D108221020114B124F1A60124BBC
:1050B0003B603368C01A114B1B68984700280AD020
:1050C0004923019A3D6023600D4B1A600D4A106020
:1050D00091221A60F7BD00220B4B23600B4B1A6024
:1050E000103232607132F4E700380140340002407F
:1050F000183801402038014018080000FC07002043
:105100001C000240200002400D000004300002405C
:105110002022034B1A600022024B1A607047C046DF
:10512000040002401C00024070B5154D2B68DB07DF
:1051300024D4144B144C1A6829235343134A2000D7
:1051400012682270124A12681112A270114A61701C
:10515000126811122271104AE17012681112A271C4
:105160001A151B136171E2712372092100F016F9FF
:105170000A220A4B60721A6093232B6070BDC046EE
:105180001C0002408C070020EC070020C80700200C
:10519000E80700207C07002078070020200002405C
:1051A00070B5394B1B78012B11D0042B12D0374B23
:1051B0001B78002B52D036490868431C0B60002333
:1051C000032844D8FF2400F065FE353C4A53FFF71E
:1051D000ABFFECE72F4D01232A68110019401A425A
:1051E000E5D12D4A2D4812680068CC335A43434319
:1051F000C8202B4C2070BE3860700238A070D014CC
:10520000D2122271DA14DB12A371264B62711B6871
:10521000E0701A14E2711A1222726372A172A01C59
:10522000092100F0CBF80C221F4BE0721A60932387
:105230002B60BCE71D4B1A68802322409B00134360
:1052400005E01B4B1B681C4080231B01234372B6E7
:10525000184A1168002900D1136062B670BD292276
:105260000D4B1B6853439B12DAB28023DB00E6E749
:1052700029220A4B1B6853431B13DAB2C023DB00FD
:10528000134300220A60E2E7C407002084070020DD
:10529000000800201C000240E80700207C070020D6
:1052A000EC0700207807002020000240C8070020FB
:1052B000CC070020880700200122074B1A60074B0B
:1052C0001968114207D0033A1A60054A054B116864
:1052D000186810601960704714100040102C0140CD
:1052E000342C01403C2C01407047000080230D4AC3
:1052F0005B0011680C480B4313600C4B19680140AC
:1053000019602021106801431160196808480140A4
:105310001960082110680143116080211A688A43CE
:105320001A60704714040048FFFFFDFF00040048A6
:10533000FFF7FFFF0A4AC307DB1713400133094A8F
:10534000FF33136008498307DB170B4020331360DA
:105350004007064BC0171840083010607047C04621
:1053600000FFFF0018040048E0FF1F00F8FF0700DF
:1053700010B51F2408490A68D3102340181806D511
:105380000020F823C0009A431043086010BD1F2876
:10539000F7DD2000F5E7C046001002400300411889
:1053A000002010B5044A8B4200D110BD1C78013397
:1053B0006040105CF7E7C046166C00080300411817
:1053C000002010B5044A8B4200D110BD1C78013377
:1053D0006040105CF7E7C046166B000810B51C0073
:1053E000884209DD904209DA029B401A1B1B584390
:1053F000511A00F0F7FD2418200010BD029CFBE7B5
:1054000010B504000020814209DB2368834201DAE1
:105410000B00934059181341C81A2060104110BD69
:10542000002303614161704730B50369C4688A1A7B
:105430006542D318AB4200DA2B00A34200DD230003
:10544000446941610C1B016803614A4341688068FB
:105450004B436043D318181830BD000070B5B54BEE
:10546000187D5C7D0200511E8A411A752200511E72
:105470008A415A759A7D511E8A41D97D9A750A00D2
:10548000551EAA41DA751A7E002A00DDC8E0012205
:105490001A765A7E002A0AD0002C00D1CAE00029D0
:1054A00000D0C7E0052A00DBBFE00522D2B25A7661
:1054B0009A7E002A00DDBFE001229A76DA7E102A69
:1054C00000DBBEE010221D7FDA76954200DA15007F
:1054D000602D00DD60255A7F1D77002A00DDB5E0D4
:1054E00001229D7F5A77954200DA1500642D00DD78
:1054F0006425DA7F9D77002A00DDACE00122DA77AF
:105500005D1CEA7F642A00DD6422EA779D1CEA7F45
:10551000002A00DDA4E00122EA77DA1CD57F642DA1
:1055200000DD6425DA1CD5771A1DD67F002296424D
:1055300003D0944201D04A424A411C1DE2775C1DCF
:10554000E47F002A00D10332944200DD14005A1D8A
:10555000D4779C1DE27F032A00DD0322E277DC1D65
:10556000E27FAA4200DA2A00642A00DD6422E277A0
:105570001A0000240832D27FA04200D16434A24233
:1055800000DD220018000830C277180028300278A9
:10559000541EA2410270E1205A8D8000824200DA3E
:1055A00002006548824200DD02001400D88DC83434
:1055B0005A85A04200DA2000604CA04200DD2000A5
:1055C0009C8D6432D885944200DA14006438844299
:1055D00000DD0400C8201A8E9C850001824200DD97
:1055E0000200588E1A86C832904200DA1000544ADF
:1055F000904200DD1000002258869A8636331878D3
:105600000200042800DD04221A704A4B022800D050
:105610009CE01A0037321278002A26DC012227E0AB
:105620001F2A00DC34E71F2232E7192A00DC3DE79D
:1056300019223BE700223AE70F2A00DC3DE70F2260
:105640003BE7302A00DC3EE730223CE7642A00DCFE
:1056500047E7642245E7642A00DC50E764224EE70E
:10566000642A00DC58E7642256E7022A00DD0200C3
:10567000D2B2180037300270180001243830027896
:10568000A243022A00DB70E0022202705A8F002A35
:105690000BD0002900D06DE02A498A4200DA0A00C6
:1056A00029498A4200DD0A0092B25A871A003C3228
:1056B0001278002A03D03C2A5EDA3C22D2B21900CA
:1056C0003C310A701A0000213D3211701A003E323E
:1056D00012788A4203D01C2A52DA1C22D2B2190054
:1056E0003E310A7019003F310A78182A00DD18226D
:1056F000FA200A70991CCA8F4000824200DD020025
:10570000CA87A12149005A5C642A00DD64225A54E8
:105710004421FF315A5C642A00DD64225A54A222DB
:1057200000215200995446210720FF315A5C024063
:105730005A5470BDC00000206C07000034080000FF
:10574000480D0000DC050000AC0D0000002203281D
:1057500000D08EE71A0037321278002A00DC5DE7AD
:105760001C2A00DC84E71C2282E7642A00DC8CE728
:1057700064228AE7002298E78C2A9FDD8C229DE72D
:10578000262AABDD2622A9E7F8B5204B1B68002BA3
:1057900001D00020F8BD1E4B1B78002BF9D172B64A
:1057A0001C4B1D4A1D4C1A601D4A1E4D1A600123D8
:1057B0005B42236003332B601B481C4B1860422361
:1057C0002B60413B22681A42FCD12B60184B06002B
:1057D0001900184A93420CD380232B6062B62468C8
:1057E0006C3B1C42D5D1521A00F0D8F943425841C3
:1057F000D0E79F1C1B88BC463380B71C012623685A
:105800003342FBD163463E00E4E7C04690070020E8
:105810000808002004200240230167450C200240B4
:10582000AB89EFCD10200240001000081420024088
:10583000C00000200802002010B572B6A32204495F
:105840005200044800F0B8F962B6FFF79DFF10BDA2
:105850006C690008C0000020064B074A1A6040220D
:10586000064B1A60064B074A1A602122064B1A6043
:105870007047C046182C0140404000001C2C0140DD
:10588000202C014044040000142C0140F0B585B0E8
:1058900000910A2203A9040000F0B4FA039D01005C
:1058A000A5423AD00B00494A0A3B0020934232D825
:1058B000474800F097FB2C000190009800282AD060
:1058C000444B1868002800D07EE0434B1E78002E21
:1058D00021D101221A70FFF7BFFF404B404A1A60E6
:1058E0006822404B1A60404B404A1A600523404AE8
:1058F00013602078651C002812D100243C4B3D4ADF
:105900001C603D4B013D1A60FFF7A6FF324B287823
:105910001C704342584105B0F0BD7D230193CCE794
:105920000300613B062B1DD8002763380721073091
:1059300000F03EFC4900042900DD01396378232B87
:1059400001D10131A51C2D4B4900CB5ABF193B4158
:10595000294A1360009B2A4A053313600022294B11
:105960001A600DE00300413B062B02D801274338A3
:10597000DCE75F281AD10023214A1360214A136013
:105980002122214B28001A6003A9173A00F03AFAA5
:10599000039BAB4216D0421E622AAED81D00019B6B
:1059A0001A495843FEF7D8FC2C00A2E72B2803D154
:1059B000002EA2D10126F7E72D289ED1002E9CD0E3
:1059C0000026F1E70120EAE70020A4E7DD0300005C
:1059D000983A00009007002008080020182C014089
:1059E000685000001C2C0140202C0140450500009F
:1059F000282C0140CF0700002C2C0140FC6A000835
:105A0000342C01403C2C0140142C0140B9520008B8
:105A1000F7B53B4B0268040000919A426FD1802396
:105A2000C2689B049A426AD1802342695B049A420D
:105A300065D1002963D0334B1B68002B5FD1324BFB
:105A40001E78002E5BD101251D70FFF705FF2F4B3F
:105A50002F4A304F1A6068222F4B1A602F4B304A62
:105A60001A60304B3E60304A1E60304B1A60212273
:105A70002F4B1A602F4B1E602369303619BA2E4BFC
:105A80004808C01800F024FA2C4B013818602C4B41
:105A90001D602C4B1D60636818BAA3681BBA019384
:105AA00023189C461A00284B18682842FCD0022074
:105AB00040421860019B002463449B1A002B18DDB0
:105AC00083231457214800990360230080334B43FC
:105AD00073435B131A333B607F2300991B1B4B43BB
:105AE000734310495B131A330B6081230132036047
:105AF000D9E7144B1C60FFF7AFFE034B1C70F7BDDA
:105B00002E736E649007002008080020182C0140B6
:105B100068500000342C01401C2C0140202C014016
:105B2000450500003C2C0140CF0700002C2C014013
:105B3000142C014028100040006CDC022C100040A6
:105B4000141000400010004010100040002C0140D4
:105B5000C317C0185840704710B50A22002100F042
:105B600051F910BD931E10B50C00222B04D900234F
:105B70001C000B70200010BD0A2A09D1002807DA8A
:105B80002D230B7001214042611800F047F9F1E725
:105B90000021F9E710B5FFF7E5FF10BD30B500248F
:105BA0000139A24201D1002005E0035D01340D5D01
:105BB000AB42F6D0581B30BD002310B59A4200D13D
:105BC00010BDCC5CC4540133F8E703008218934243
:105BD00000D1704719700133F9E703000A78180003
:105BE0001A7001310133002AF8D17047F0B5050071
:105BF00000240327094E2A5DB35C3B40012B00D1F2
:105C000020320B5DF05C3840012800D12033D01ADF
:105C10009A4202D10134002BEDD1F0BD3C6D000859
:105C2000F0B50500002A14D0501E012A1CD02C000B
:105C30000A001600270036780132013413002500CF
:105C40003E70002E0DD001380028F2D100222A70BB
:105C500000E00B001A000132501E007813000028EB
:105C6000F9D1581A0138F0BD0B00EFE70023C25CF0
:105C70000133002AFBD1581E704710B502000023E3
:105C8000006800F001F810BDF0B5002802D11068DE
:105C9000002813D0040020000E0005780134377866
:105CA000002F04D1002D0FD12800156006E0013629
:105CB000BD42F4D1002BEED114600370F0BD2F0073
:105CC0000FE00133002E04D1230001341D7827009A
:105CD0000B001E78B542F4D1002DF0D00023013C1A
:105CE00023701760EAE70000F0B587B01E0005904A
:105CF00001910292012B45D00B00242E42D83F4A3D
:105D0000082194461A00604614780133005D1D0096
:105D100007000F400842F5D12D2C3AD101271C78FD
:105D2000951C002E65D0102E09D1302C07D12022D1
:105D30002B789343582B57D110266C780235304B73
:105D40003100FB181800039300F048F900230122EA
:105D500084461800049152422100303909291DD887
:105D60000C00A64228DD002B24DB1300844506D35B
:105D700002D10499A14202DB0123704320182C7840
:105D80000135E9E700F080F816230360002007B032
:105D9000F0BD2B2CC5D11C78951CC2E721004139E0
:105DA000192901D8373CDCE721006139192903D8CA
:105DB000573CD6E71300E2E7002B09DA2223059AC5
:105DC00003981360029B002BE1D06B1E019307E048
:105DD000002F00D04042029A002AD8D0002BF4D1E4
:105DE000029B019A1A60D2E73024002EA7D1083610
:105DF000A5E7302C9BD00A26A1E7C0463C6D0008E1
:105E0000FFFFFF7F10B513000A0001000248006881
:105E1000FFF76AFF10BDC0465C020020F0B50C0021
:105E200016008DB025220700164902A8FFF7C4FE10
:105E3000621E0092B31E02AA00250192222B04D9F1
:105E400025702C0020000DB0F0BD3800310000F0AE
:105E5000C5F80B00019A2900D35C009A013553550F
:105E60003B0007009E42F0D90023220063550B003F
:105E7000C81A8342E6DD1078E55C1570E054013203
:105E8000013BF5E7166D0008014B18687047C046E6
:105E90005C02002002B4714649084900095C4900CF
:105EA0008E4402BC7047C04603B4714649084000A6
:105EB0004900095E49008E4403BC704703B4714633
:105EC000490840004900095A49008E4403BC704704
:105ED000002243088B4274D303098B425FD3030A29
:105EE0008B4244D3030B8B4228D3030C8B420DD33C
:105EF000FF22090212BA030C8B4202D312120902CA
:105F000065D0030B8B4219D300E0090AC30B8B4207
:105F100001D3CB03C01A5241830B8B4201D38B03B5
:105F2000C01A5241430B8B4201D34B03C01A52415A
:105F3000030B8B4201D30B03C01A5241C30A8B429D
:105F400001D3CB02C01A5241830A8B4201D38B0288
:105F5000C01A5241430A8B4201D34B02C01A52412C
:105F6000030A8B4201D30B02C01A5241CDD2C3099E
:105F70008B4201D3CB01C01A524183098B4201D31A
:105F80008B01C01A524143098B4201D34B01C01A05
:105F9000524103098B4201D30B01C01A5241C3087D
:105FA0008B4201D3CB00C01A524183088B4201D3EC
:105FB0008B00C01A524143088B4201D34B00C01AD8
:105FC0005241411A00D20146524110467047FFE744
:105FD00001B5002000F0F0F802BDC0460029F7D05E
:105FE00076E7704703460B437FD4002243088B4279
:105FF00074D303098B425FD3030A8B4244D3030B50
:106000008B4228D3030C8B420DD3FF22090212BA14
:10601000030C8B4202D31212090265D0030B8B4290
:1060200019D300E0090AC30B8B4201D3CB03C01A7A
:106030005241830B8B4201D38B03C01A5241430B55
:106040008B4201D34B03C01A5241030B8B4201D345
:106050000B03C01A5241C30A8B4201D3CB02C01AB0
:106060005241830A8B4201D38B02C01A5241430A28
:106070008B4201D34B02C01A5241030A8B4201D317
:106080000B02C01A5241CDD2C3098B4201D3CB01BE
:10609000C01A524183098B4201D38B01C01A52416D
:1060A00043098B4201D34B01C01A524103098B4271
:1060B00001D30B01C01A5241C3088B4201D3CB005C
:1060C000C01A524183088B4201D38B00C01A52413F
:1060D00043088B4201D34B00C01A5241411A00D2EF
:1060E00001465241104670475DE0CA0F00D0494258
:1060F000031000D34042534000229C4603098B42C8
:106100002DD3030A8B4212D3FC22890112BA030A4F
:106110008B420CD3890192118B4208D389019211D1
:106120008B4204D389013AD0921100E08909C30956
:106130008B4201D3CB01C01A524183098B4201D358
:106140008B01C01A524143098B4201D34B01C01A43
:10615000524103098B4201D30B01C01A5241C308BB
:106160008B4201D3CB00C01A524183088B4201D32A
:106170008B00C01A5241D9D243088B4201D34B0045
:10618000C01A5241411A00D20146634652415B1087
:10619000104601D34042002B00D549427047634668
:1061A0005B1000D3404201B5002000F005F802BDAD
:1061B0000029F8D016E770477047C046FEE77047E1
:1061C00010B5164B164A17498B4218D30021164AB0
:1061D000934217D38023154A9B001168144C0B433C
:1061E0001360144B9C420FD3134C144B9C420ED3A0
:1061F000FEF77EF9124C134B9C420BD310BD01CA23
:1062000001C3E1E702C3E3E708CC9847E9E708CC1C
:106210009847EAE708CC9847EDE7C0460802002017
:106220003C6E0008C00200200C08002014ED00E0C5
:106230003C6E00083C6E00083C6E00083C6E000896
:106240003C6E00083C6E0008014B024A1A60FEE7F3
:106250000CED00E00400FA05044A43099B009B187A
:106260001F2210401E3A82401A60704700E100E091
:1062700010B51F2812D90F2318400438C0B2830864
:10628000084A9B001824C0002040E7348440814025
:106290009B181A68A2431143196010BD8308024A73
:1062A0009B00EFE718ED00E000E400E051416100E1
:1062B000A000A300A600A800AB00AE00B100B30090
:1062C000B600B900BC00BF00C100C400C700C900CF
:1062D000CC00CF00D100D400D700D900DC00DF0013
:1062E000E100E400E600E900EB00EE00F000F2005F
:1062F000F500F700F900FC00FE00000103010501B4
:10630000070109010B010D010F0111011301150115
:10631000170119011B011C011E012001210123018C
:1063200025012601280129012B012C012D012F0116
:1063300030013101320133013401350136013701B9
:10634000380139013A013B013B013C013D013D016E
:106350003E013E013E013F013F013F01400140013E
:1063600040014001400140014001400140013F0126
:106370003F013F013E013E013E013D013D013C0127
:106380003B013B013A013901380137013601350142
:10639000340133013201310130012F012D012C0173
:1063A0002B012901280126012501230121012001BA
:1063B0001E011C011B011901170115011301110117
:1063C0000F010D010B010901070105010301000186
:1063D000FE00FC00F900F700F500F200F000EE000E
:1063E000EB00E900E600E400E100DF00DC00D9009A
:1063F000D700D400D100CF00CC00C900C700C40032
:10640000C100BF00BC00B900B600B300B100AE00CF
:10641000AB00A800A600A300A0009D009A00980071
:10642000950092008F008D008A0087008400810013
:106430007F007C0079007700740071006F006C00B1
:1064400069006700640061005F005C005A0057004B
:106450005500520050004E004B00490047004400D8
:10646000420040003D003B0039003700350033005A
:1064700031002F002D002B002900270025002400CB
:10648000220020001F001D001B001A00180017002A
:10649000150014001300110010000F000E000D0075
:1064A0000C000B000A0009000800070006000500A8
:1064B00005000400030003000200020002000100C6
:1064C00001000100000000000000000000000000CA
:1064D00000000000000001000100010002000200B5
:1064E0000200030003000400050005000600070089
:1064F000080009000A000B000C000D000E000F0040
:1065000010001100130014001500170018001A00E5
:106510001B001D001F002000220024002500270072
:1065200029002B002D002F003100330035003700EB
:1065300039003B003D004000420044004700490054
:106540004B004E0050005200550057005A005C00AE
:106550005F0061006400670069006C006F007100FB
:106560007400770079007C007F0081008400870040
:106570008A008D008F009200950098009A009D007F
:106580002E00300020090D0A0055736167653A0A34
:10659000696E666F0A73686F770A676574203C706E
:1065A0006172616D3E0A736574203C706172616D49
:1065B0003E203C76616C75653E0A736176650A72B1
:1065C000657365740A706C6179203C6D75736963DD
:1065D0003E205B3C766F6C756D653E5D0A7468723B
:1065E0006F74203C76616C75653E0A626565700A61
:1065F0000045534361706533322072657600205B3D
:10660000005D0A54656D703A2000432C2065787453
:106610002000430A566F6C743A2000560A43757284
:10662000723A2000410A4373756D3A20006D41684B
:106630000A4552504D3A200061726D0064616D70E0
:1066400000726576646972006272757368656400D1
:1066500074696D696E670073696E655F72616E67FC
:10666000650073696E655F706F776572006672654D
:10667000715F6D696E00667265715F6D617800644F
:106680007574795F6D696E00647574795F6D61789A
:1066900000647574795F7370757000647574795FE8
:1066A00072616D7000647574795F72617465006405
:1066B0007574795F6472616700647574795F6C6F7B
:1066C000636B007468726F745F6D6F6465007468EB
:1066D000726F745F726576007468726F745F627255
:1066E0006B007468726F745F736574007468726FA6
:1066F000745F63616C007468726F745F6D696E00C3
:106700007468726F745F6D6964007468726F745F2F
:106710006D617800616E616C6F675F6D696E0061BD
:106720006E616C6F675F6D617800696E7075745F24
:106730006D6F646500696E7075745F63686964008D
:1067400074656C656D5F6D6F64650074656C656D17
:106750005F706869640074656C656D5F706F6C650F
:10676000730070726F745F7374616C6C0070726F21
:10677000745F74656D700070726F745F73656E73B3
:106780000070726F745F766F6C740070726F745FFC
:1067900063656C6C730070726F745F637572720006
:1067A0006D7573696300766F6C756D650062656108
:1067B000636F6E00626563006C6564004F4B0A0096
:1067C0004552524F520A0068656C7000696E666FE0
:1067D0000073686F77006765740073617665007297
:1067E0006573657400706C6179007468726F740011
:1067F0006265657000000000C7670008CC6700088C
:10680000D1670008D6670008E8660008DA67000864
:10681000DF670008E5670008EA670008F06700081E
:1068200000000000386600083C6600084166000869
:10683000486600085066000857660008626600084F
:106840006D660008766600087F66000888660008A6
:10685000916600089B660008A5660008AF66000800
:10686000B9660008C3660008CE660008D86600084E
:10687000E2660008EC660008F6660008006700089B
:106880000A670008146700081F6700082A670008E5
:1068900035670008406700084B6700085667000826
:1068A000626700086D670008776700088167000865
:1068B0008B67000896670008A0670008A6670008B5
:1068C000AD670008B4670008B86700080000000062
:1068D000191B12131D1516171A090A0B1E0D0E0F80
:1068E0004743006336004623324532443243320088
:1068F0004723412347234123472332004723412392
:10690000472341234623324723320047234123476D
:106910002341234532462332472332004723412374
:10692000472341234432453246233247233200472E
:106930002341234723412343324432453246233205
:106940004723320045470046410047420041422369
:106950000061444745000000446900084769000899
:106960004A6900084D69000851690008EA320E02C0
:1069700049464C49474854310000000000000000DF
:1069800001010000100008183001640F001E000013
:10699000000064000100E803DC05D0076400800CFF
:1069A000000000000E00000000000000000064660F
:1069B0006123000000000000000000000000000053
:1069C00000000000000000000000000000000000C7
:1069D00000000000000000000000000000000000B7
:1069E00000000000000000000000000000000000A7
:1069F0000000000000000000000000000000000097
:106A00000000000000000000000000000000000086
:106A10000000000000000000000000000000000076
:106A20000000000000000000000000000000000066
:106A30000000000000000000000000000000000056
:106A40000000000000000000000000000000000046
:106A50000000000000000000000000000000000036
:106A60000000000000000000000000000000000026
:106A70000000000000000000000000000000000016
:106A80000000000000000000000000000000000006
:106A900000000000000000000000000000000000F6
:106AA000000000000000000000000000000019329B
:106AB000000035192B321E2CE3680008ED68000831
:106AC000EB680008E9680008E6680008F06800085C
:106AD000FC6800080B6900081C6900082F690008A1
:106AE0000000000001020102030205020602020288
:106AF000700B000410020002300B0005B73B5D383C
:106B000033353832652FBC2C3A2ADB279E25822369
:106B10008321A11FDB1D00D57FAAFE2B815429FCF8
:106B20005683D702A87D52872DF8AC79D3067BAE69
:106B300004D18550FA2FA471DB0E5A8F25F08D58A1
:106B4000F22773A60CD9F623895C08DD77A2DF0A49
:106B5000A07521F45E8B9D48E23763B61CC9B46111
:106B6000CB1E4A9F35E0CF1AB06531E44E9BE63329
:106B7000994C18CD67B239EC4693C712B86D10C561
:106B80006FBAEE3B91446BBE14C19540EA3F429709
:106B90003DE8BC69C316EF3A904511C46EBBC613FD
:106BA000B96C38ED4792BD68C21743963CE99441F1
:106BB000EB3E6ABF15C04B9E34E1B560CA1F62B799
:106BC0001DC89C49E33619CC66B3E732984D30E5D1
:106BD0004F9ACE1BB16472A70DD88C59F3265B8EE9
:106BE00024F1A570DA0F20F55F8ADE0BA17409DCB1
:106BF00076A3F722885DD603A97C28FD5782FF2A59
:106C0000805501D47EAB8451FB2E7AAF05D0AD7890
:106C1000D20753862CF900070E091C1B1215383FAA
:106C2000363124232A2D70777E796C6B6265484F4C
:106C3000464154535A5DE0E7EEE9FCFBF2F5D8DF3C
:106C4000D6D1C4C3CACD90979E998C8B8285A8AFAC
:106C5000A6A1B4B3BABDC7C0C9CEDBDCD5D2FFF89C
:106C6000F1F6E3E4EDEAB7B0B9BEABACA5A28F880C
:106C7000818693949D9A2720292E3B3C35321F18FC
:106C8000111603040D0A5750595E4B4C45426F686C
:106C9000616673747D7A898E878095929B9CB1B66C
:106CA000BFB8ADAAA3A4F9FEF7F0E5E2EBECC1C6CC
:106CB000CFC8DDDAD3D4696E676075727B7C5156BC
:106CC0005F584D4A4344191E171005020B0C21262C
:106CD0002F283D3A33344E49404752555C5B76711C
:106CE000787F6A6D64633E39303722252C2B06018C
:106CF000080F1A1D1413AEA9A0A7B2B5BCBB96917C
:106D0000989F8A8D8483DED9D0D7C2C5CCCBE6E1EB
:106D1000E8EFFAFDF4F330313233343536373839B1
:106D20006162636465666768696A6B6C6D6E6F70DB
:106D30007172737475767778797A0000202020203C
:106D4000202020202028282828282020202020201B
:106D500020202020202020202020202088101010FB
:106D60001010101010101010101010100404040453
:106D700004040404040410101010101010414141C8
:106D80004141410101010101010101010101010133
:106D900001010101010101101010101010424242C6
:106DA0004242420202020202020202020202020203
:106DB0000202020202020210101010200000000065
:106DC00000000000000000000000000000000000C3
:106DD00000000000000000000000000000000000B3
:106DE00000000000000000000000000000000000A3
:106DF0000000000000000000000000000000000093
:106E00000000000000000000000000000000000082
:106E10000000000000000000000000000000000072
:106E20000000000000000000000000000000000062
:0C6E300000000000000000000000000056
:106E3C00FFFFFFFFFFFFFFFF0000FFFF0000FFFF52
:106E4C00FFFF0000FFFF0000FFFFFFFF0000FFFF40
:106E5C000000FFFF0000FFFFFFFFFFFF000000002E
:106E6C0000000000FFFFFFFFFFFFFFFFFFFFFFFF22
:106E7C00FFFFFFFFFFFFFFFFFFFFFFFFFFFFFFFF16
:106E8C00E40C000060020020000000000000000084
:106E9C0000000000000000000000000000000000E6
:106EAC0000000000000000000000000000000000D6
:106EBC0000000000000000000000000000000000C6
:106ECC0000000000000000000000000000000000B6
:106EDC0000000000000000000000000000000000A6
:086EEC0000000000000000009E
:04000005080061C1CD
:00000001FF
